:1000000001280C3085000030860083160030850002
:10001000FF3086000030810083123E2003012A2039
:10002000851110302A203B2030302A203B20203000
:100030002A203B2060302A203B2040302A203B20D1
:10004000C0302A203B2080302A203B2090302A20BC
:100050003B2011288E0008308F0085108E1B8514E0
:100060008E0D00000514000005108F0B2D280515BE
:1000700000000511080001308C004128F4308C008C
:1000800041288D0100000000000000000000000079
:1000900000000000000000000000000000008D0BC8
:0800A00042288C0B41280800E6
:02400E00F13F80
:00000001FF
